:100000000C94A2020C94DA020C94DA020C94DA0238
:100010000C94DA020C94DA020C94DA020C94DA02F0
:100020000C94DA020C94DA020C942A210C946620C7
:100030000C94CB250C94DA020C94DA020C94DA02BC
:100040000C94DA020C947E140C94DA020C94DA020A
:100050000C94DA020C948A250C94DA020C94DA02DD
:100060000C94DA020C94DA020C94DA020C94DA02A0
:100070000C94DA020C94DA020C94DA020C94DA0290
:100080000C94DA020C94DA020C94DA020C94DA0280
:100090000C94DA020C94DA020C94DA020C94DA0270
:1000A0000C94DA020C94DA020C94DA02E306E3060A
:1000B000150715078707A3073A093A09AE078C0801
:1000C0009D089D087F1EA61E3E20A61E3E20EE1EF9
:1000D000111F3E200020132000047F3F1F643214B4
:1000E0006432141E05FB1E140A052B0014001A00AE
:1000F0000800150017001C0018000C001200130067
:100100002A00290004001600070009000A000B005D
:100110000D000E000F0033002800E1001D001B0041
:1001200006001900050011001000360037003800E5
:100130005200E000E300E2002F002D002C410000FF
:100140002E003000500051004F00AA00A90000000E
:1001500000000000000000000000000000004E0051
:100160004B0035001E001F0020002100220023004C
:1001700024002500260027000100010001000100E5
:100180000100010001000100010001000100010067
:100190000100010001000100010001000100010057
:1001A0000100010001000100010001000100010047
:1001B00001002A00010000004C0001000100310094
:1001C000010001000100000000000000000000002C
:1001D0000000000000000100010000010101010118
:1001E00001010101020202020202020202030303F0
:1001F00003030303030404040404040405050505C0
:10020000050606060606070707070708080808097F
:100210000909090A0A0A0B0B0B0C0C0C0D0D0D0E2B
:100220000E0E0F0F0F1010111111121213131414C0
:10023000151516161717181819191A1A1B1B1C1D35
:100240001D1E1E1F2020212222232424252626278E
:100250002829292A2B2C2D2D2E2F303132323334C0
:1002600035363738393A3B3C3D3E3F4041424344C6
:1002700045464748494A4C4D4E4F505153545556A8
:1002800058595A5B5D5E5F616264656668696B6C54
:100290006D6F7072737577787A7B7D7E80828385CF
:1002A00087888A8C8E8F91939596989A9C9EA0A20F
:1002B000A3A5A7A9ABADAFB1B3B5B7BABCBEC0C219
:1002C000C4C6C9CBCDCFD1D4D6D8DBDDDFE2E4E7DD
:1002D000E9EBEEF0F3F5F8FAFDFFFFAA7F554005D4
:1002E000010902A10185020901A1000509190129DD
:1002F00008150025019508750181020501093009DD
:10030000311581257F9502750881060938158125EB
:100310007F950175088106050C0A38021581257F35
:10032000950175088106C0C005010980A1018503FA
:1003300019012AB700150126B70095017510810033
:10034000C0050C0901A101850419012AA0021501AB
:1003500026A002950175108100C005010906A101C2
:100360008506050719E029E715002501950875019F
:1003700081020507190029EF1500250195F0750187
:10038000810205081901290595057501910295015C
:1003900075039101C005010906A101050719E029AE
:1003A000E715002501950875018102950175088101
:1003B000010507190029FF150026FF00950675089D
:1003C000810005081901290595057501910295011E
:1003D00075039101C009023B00020100A0FA090463
:1003E0000000010301010009211101000122400068
:1003F0000705810308000109040100010300000052
:1004000009211101000122B6000705820320000125
:100410001201000200000008EDFE60600100010210
:1004200000010E035400650074007200690073003F
:1004300000000C03460065006E0067007A000000B3
:10044000040309042223252628292A2C2D2F3032A3
:10045000333536383A3B3D3E4042434547494A4CA6
:100460004E5051535557595A5C5E606264666869D4
:100470006B6D6F71737577797B7D7F8183858789DC
:100480008A8C8E90929496989A9C9E9FA1A3A5A7E1
:10049000A8AAACAEAFB1B3B4B6B8B9BBBCBEBFC10D
:1004A000C2C3C5C6C7C9CACBCCCDCED0D1D2D2D398
:1004B000D4D5D6D7D7D8D9D9DADADBDBDBDCDCDCAC
:1004C000DCDCDDDDDDDDDCDCDCDCDCDBDBDBDADA6F
:1004D000D9D9D8D7D7D6D5D4D3D2D2D1D0CECDCCE6
:1004E000CBCAC9C7C6C5C3C2C1BFBEBCBBB9B8B6FB
:1004F000B4B3B1AFAEACAAA8A7A5A3A19F9E9C9A86
:1005000098969492908E8C8A89878583817F7D7B53
:1005100079777573716F6D6B6968666462605E5C34
:100520005A5957555351504E4C4A494745434240FA
:100530003E3D3B3A3836353332302F2D2C2A292890
:100540002625232211241FBECFEFDAE0DEBFCDBF68
:1005500004B603FE18C080917F0490918004A0919E
:100560008104B09182048730904BA740B04B59F47E
:1005700010927F04109280041092810410928204E1
:10058000E0E0F8E3099512E0A0E0B1E0E8EAFDE57B
:1005900002C005900D92A235B107D9F724E0A2E57B
:1005A000B2E001C01D92AF37B207E1F70E94C40A62
:1005B0000C94D22E0C9400001F93CF93DF93CDB7F1
:1005C000DEB767970FB6F894DEBF0FBECDBF4B8B7B
:1005D0005C8B6D8B7E8B8F8B611110921E0386E07E
:1005E0009E01235F3F4FD901E82F1D92EA95E9F75D
:1005F00095E0FE017396D90101900D929A95E1F76D
:100600009C894E895F897B897D879E876F87598BFF
:10061000488BF901DE01179601900D928A95E1F75A
:10062000CE0107960E94DB2781113EC086E0FE01C5
:100630003796DE01119601900D928A95E1F7FF81C0
:10064000E8856A857B856115710531F0EF3F31F4EE
:1006500081E0FF3F19F403C081E001C080E080FD2C
:1006600023C02091CB0230E0C90101968770992701
:100670004091FC0250E08417950779F1F983EA83F1
:100680007D836C8396E0929FD001939FB00D1124DF
:10069000A453BD4FFE01319601900D929A95E1F75A
:1006A0008093CB020E94391C16E08091FC0290914D
:1006B000CB028917F9F0189FC001112484539D4F74
:1006C0000E94DB278823B1F08091FC0290E0019624
:1006D000877099278093FC02E8CF0E942D2A109200
:1006E000CB021092FC02E5ECF2E086E0DF011D9205
:1006F0008A95E9F767960FB6F894DEBF0FBECDBFB7
:10070000DF91CF911F9108958F929F92AF92BF92E8
:10071000CF92DF92EF92FF920F931F93CF93DF93CD
:10072000CDB7DEB72A970FB6F894DEBF0FBECDBFA8
:10073000FC010081D18083819481892B39F01FEFE6
:10074000D11206C091E00F3F19F403C091E001C03F
:1007500090E090FDB6C67F0185E0DE01169601901F
:100760000D928A95E1F7F70122818E819F812223E4
:1007700049F00E944627182F682F8E819F810E9482
:10078000A82903C00E947C29182F2CE3129FF00196
:1007900011243CE0D39EE00DF11D1124E00FF11D6A
:1007A000EE0FFF1FE651FF4F05911491043C8CE5BD
:1007B000180749F480913C04869590E09093B2012B
:1007C0008093B10136C00D319CE5190741F4F70162
:1007D0008281882309F4A2C10E94B82B9FC50E31E3
:1007E000FCE51F0741F4F7018281882309F496C1D3
:1007F0000E949E2B93C50F31FCE51F0749F4F701BA
:1008000082818823D9F080916B0380FDF1CFE4CF02
:100810000A32FCE51F0769F4F7018281882371F031
:1008200010926D0364E070E080E091E00E94F11CA2
:1008300075C50B32FCE51F0779F370C1F7018281A2
:10084000882309F4D0C1109246040430FDE51F0747
:1008500058F40B3F2CE5120780F4C80182509C45E8
:10086000449708F0AAC109C002363DE5130729F0F4
:10087000063A8DE5180709F0A0C10E94211B90934C
:1008800053048093520401319CE5190709F4CEC04A
:1008900008F045C00930FCE51F0709F4A5C000F5C4
:1008A00005303CE5130709F48DC078F403309CE56E
:1008B000190709F47FC008F081C002301C4509F017
:1008C0001DC180915204816017C107302CE51207C9
:1008D00009F482C008F084C08091520480610CC188
:1008E0000D308CE5180709F48DC070F40B30ECE581
:1008F0001E0709F47FC008F081C08091520488600F
:10090000846080935204B3C00F302CE5120709F4C1
:1009100085C008F087C080915204877FEDC00E3FEC
:100920008CE5180709F476C008F50531ECE51E07DB
:1009300009F48EC068F403312CE5120709F47AC07B
:1009400008F0B8C00E942D2A809152048F77D4C03D
:100950000C3F8CE51807D1F108F058C00B3F1C453F
:1009600009F0CCC080915304816033C00230FDE5B2
:100970001F0709F4ABC070F401153DE5130709F436
:1009800060C008F07EC080915304826081608093D3
:10099000530484C002369DE5190709F49DC0063A48
:1009A000EDE51E0709F4A2C003301D4509F0A6C0FD
:1009B00060E08DC08091520482609EC0809152049C
:1009C00084609AC080915204886096C080915304DC
:1009D00082608093530492C08091520480628CC0E4
:1009E00080915204806488C00E942D2A8091520414
:1009F000806882C0809152048E7F7EC080915204B4
:100A00008D7F7AC0809152048B7F76C08091530491
:100A10008E7FDFCF809153048D7FDBCF8091520496
:100A20008F7E6AC0809152048F7D66C0809152048F
:100A30008F7B62C080915204877F8B7F80935204AA
:100A40001BC0809153048D7F8E7F809353042BC0F5
:100A50008091520482FB222720F991E0922790FB9B
:100A600082F990FB83F980935204992329F064E082
:100A700070E080E691E01BC062E070E080E391E00E
:100A800016C080915304982F909591708E7F892B7A
:100A900090FB81F980935304992329F064E070E07E
:100AA00080E491E004C062E070E080E291E00E94A6
:100AB000F11C24C00E942D2A8091520487FB22271A
:100AC00020F991E0922790FB87F916C061E08EE053
:100AD00090E00E94242C12C08091520484FB2227B3
:100AE00020F991E0922790FB84F906C0809152048E
:100AF000982F909590FB80F9809352046091520456
:100B00001091530484E090E00E94242C612F82E233
:100B100090E00E94242C0E942D2A00C4043F2CE562
:100B2000120749F406E221EE40EE64EF7CE5C701CE
:100B30000E948926F3C3053F3CE51307F8F4093DFD
:100B40008CE5180731F407E225EE45EE69ED7CE50A
:100B5000EECF0A3D9CE5190731F408E221E045EEAD
:100B60006AED7CE5E4CF083DECE51E0709F066CEB2
:100B700006E221EE41EE68ED7CE5D9CF063FFCE5CB
:100B80001F0731F406E221EE42EE66EF7CE5CFCF9F
:100B9000063F2CE5120730F407E225EE44EE65EF40
:100BA0007CE5C5CF073F3CE5130709F047CE07E2D8
:100BB00025EE46EE67EF7CE5BACF06318CE51807E7
:100BC00021F580911F038A7A91E009F490E09093D7
:100BD0005402882311F065E301C069E285EA92E0DE
:100BE0000E941C260FC00631FCE51F0709F073C0E8
:100BF00080915402882309F4B4C365E385EA92E046
:100C00000E94F4250E94AA1B89C30B353DE51307FA
:100C100009F45BC058F401159CE51907C1F00F3DBC
:100C20001C4509F074C00E94321B78C30C35FDE5E9
:100C30001F0709F44CC00D351D4509F068C08091AF
:100C4000530482FB882780F991E0892741C00E94E4
:100C50002D2A0E94BF258C0163E070E080E891E0BE
:100C60000E94F11CC8010E94B0258A3F910538F40A
:100C70008FE99FE00197F1F700C00000F3CF0E94D9
:100C8000772B81E08093E00080E28093D80010927F
:100C9000C900EFE1FEE43197F1F700C0000087E002
:100CA00090EBDC0180937F0490938004A0938104F7
:100CB000B09382049CE088E10FB6F894A8958093E5
:100CC00060000FBE90936000FFCF81E001C080E024
:100CD0000E941C1C1CC080911F0382720D3C2CE5DD
:100CE000120709F4D0C308F002C3073C9CE51907BA
:100CF00009F4B5C308F045C3043CFCE51F0709F43B
:100D0000A4C308F030C3033C1C4509F47AC3F701BF
:100D100082810081D180882359F0802F9D2D0E94EF
:100D20004627182F682F802F9D2D0E94A82905C0C7
:100D3000802F9D2D0E947C29182F2CE3129FF001FB
:100D400011243CE0D39EE00DF11D1124E00FF11DB4
:100D5000EE0FFF1FE651FF4F859194910E94871976
:100D60008C01982EF701D280A580A2943FE0A322A7
:100D70008091FD028770B9F0DD20A9F0812F807F7E
:100D8000803421F080E2800F883068F08091530435
:100D900082FD09C082E00E94FF1B8091FD028770E6
:100DA000CC24C3948111C12CB12EB2949FE0B922FE
:100DB0008B2D90E08C30910508F05CC2FC01EA5A62
:100DC000FF4F0C94752E812F807F1F70882311F0A8
:100DD0001295107FDD20B9F0112309F438C280E2AA
:100DE000800F883010F0911006C080911F03182BDF
:100DF00010931F0305C080911E03182B10931E0330
:100E00000E94AA1B24C2802F0E94532A112309F496
:100E100031C2005E083078F1992069F11095809117
:100E20001E03182310931E0329C0812F807F1F707B
:100E3000803211F01295107F992021F0F1E09F1679
:100E4000D9F149C08091530482FF1BC0DD2069F0B5
:100E5000112339F080911F03182B10931F030E9458
:100E6000AA1B80E00E94B32A05C280E00E94532A98
:100E7000112309F4FFC1812F0E94A31B0E94AA1B0A
:100E8000F9C1DD2081F080912003AA2051F001E01A
:100E9000A01207C0182B181709F4ECC110932003F7
:100EA000E9C1812B10C0AA2021F021E0A21609F48B
:100EB000E1C10E949D1B27C0DD2041F035E03A15BD
:100EC00008F4D8C1812F0E94492AD4C184E08A1530
:100ED00008F4D0C118C0DD2049F0AA2099F3F70129
:100EE000858180FFB4C18F708583ECCFAA2059F033
:100EF000093309F0BCC1FFEF17EE23E0F1501040B9
:100F00002040E1F7B2C1812F0E94422AB3C1812F54
:100F100086958695837019F0813059F0ABC1DD203C
:100F200019F0C801937002C080E090E00E9467262B
:100F3000A7C1DD2019F0C801937002C080E090E0E5
:100F40000E9451269DC1802FDD2019F00E94481378
:100F500002C00E948F120E94651292C1812F83707D
:100F600009F069C0D1108AC1902F9295969597701B
:100F7000990F990F802F8F70882E912CA12CB12C56
:100F8000092E04C0880C991CAA1CBB1C0A94D2F719
:100F900004FF12C04FE050E060E070E004C0440F76
:100FA000551F661F771F9A95D2F7DB01CA018095FE
:100FB0009095A095B09503C080E090E0DC01169577
:100FC0001695412F4370423019F1C8F40091210366
:100FD000109122032091230330912403413059F0D2
:100FE00088299929AA29BB29BC01CD016023712335
:100FF000822393230AC0802A912AA22AB32ABC0101
:10100000CD01682979298A299B290E94232A36C182
:1010100088299929AA29BB2900912103109122032B
:101020002091230330912403BC01CD016027712757
:1010300082279327EACFDD2019F0812F817001C02C
:101040008695882309F41AC1902F929596959770EA
:10105000990F990F802F8F70882E912CA12CB12C75
:10106000092E04C0880C991CAA1CBB1C0A94D2F738
:1010700004FF12C04FE050E060E070E004C0440F95
:10108000551F661F771F9A95D2F7DB01CA0180951D
:101090009095A095B09503C080E090E0DC01169596
:1010A0001695412F43704230D9F068F500917802CF
:1010B0001091790220917A0230917B02413059F0EF
:1010C00088299929AA29BB29BC01CD016023712354
:1010D000822393231EC0802A912AA22AB32A13C0F6
:1010E00088299929AA29BB290091780210917902AF
:1010F00020917A0230917B02BC01CD0160277127DB
:101100008227932706C0BC01CD01682979298A2945
:101110009B290E94D329B2C01F70DD2039F0812F96
:101120000E94022A802F0E94492AA8C0802F0E9474
:10113000422A812F0E94DD29A1C0802F32EF931611
:1011400009F443C0391538F090EF991659F0E1EFE2
:101150009E16B1F177C0F3EF9F16F1F124EF9216CE
:1011600059F170C0DD2019F134E03A1508F482C05D
:101170001F7181E090E0A0E0B0E0AC01BD0104C0CF
:10118000440F551F661F771F1A95D2F7809178027A
:1011900090917902A0917A02B0917B028A019B0121
:1011A000082719272A273B27C901B80129C025E0AC
:1011B0002A1508F45FC0DCCF8091530482FF23C05E
:1011C000DD2029F0812F8F7130C0DD20D9F3812FF0
:1011D0008F710E94DD294EC0DD2079F01F7181E002
:1011E00090E0A0E0B0E0BC01CD0104C0660F771F25
:1011F000881F991F1A95D2F703C060E070E0CB01F9
:101200000E94D32937C0DD2099F01F71812F0E94E1
:10121000022A8091530482FD07C038E0139FC00169
:10122000112483608093FD02812F0E94022A22C034
:1012300081E00E94FF1B81E08A15E0F482E00E94B9
:10124000FF1B18C0DD2029F0AA2009F4BBCF802F96
:1012500009CEAA2009F4BBCF893349F49FEFE7EE0A
:10126000F3E09150E040F040E1F700C00000802F33
:101270000E94532A88EF8B0D843010F40E947D2643
:10128000CC20A9F08091FD0280FD11C0F7011282EF
:101290008595859585950E94022AC7010E94840341
:1012A0008091FD028595859585950E94DD2985E0D3
:1012B000F701DE01119601900D928A95E1F789817F
:1012C0009A810E947C299A810CE3809FF00111246D
:1012D0001CE0919FE00DF11D11248981E80FF11DA3
:1012E000EE0FFF1FE651FF4F85919491EAC0023D3A
:1012F0002CE5120709F4D6C008F465C0053D2CE5BD
:10130000120709F4D5C008F471C0063DECE51E07CC
:1013100009F4D3C00E351D4509F0F9CC8091FD02CA
:10132000877009F4CEC0F7018281882309F4C9C00F
:101330008091530482FDC5C082E02A960FB6F894CE
:10134000DEBF0FBECDBFDF91CF911F910F91FF90F8
:10135000EF90DF90CF90BF90AF909F908F900C94C4
:10136000FF1B69E24BCC053C9CE5190709F472C0F0
:10137000063C1C4509F0CBCC42E052E16BE072E147
:1013800086C00A3CFCE51F0709F473C070F4083CF2
:101390003CE5130709F468C0093C1C4509F0B7CCCB
:1013A00046EF51E16AEE71E172C00B3CECE51E07BD
:1013B00009F464C00C3C1C4509F0A9CC46E550E199
:1013C00067E670E164C00F3C8CE5180709F464C05F
:1013D00008F460C0003DECE51E0709F460C0013D63
:1013E0001C4509F094CC6EE089E064C0033D8CE5B7
:1013F000180709F45AC0043D1C4509F088CC88E15F
:101400005DC080913C0480FF1BC08E7F80933C04B4
:1014100060913C0470913D0480913E0490913F04A2
:101420000E9444101092A4020FEF10E722E0015036
:1014300010402040E1F700C000000E94EA0F6ECF8C
:10144000816080933C04869539C042E552E16BE5AA
:1014500072E11DC04BE552E162E572E118C04BE05C
:1014600052E162E072E113C04AEE51E166EF71E1D0
:101470000EC042ED51E16EED71E109C04EED51E15A
:1014800062ED71E104C047E650E166E570E10E945B
:10149000252744CF81E012C065E082E00BC068E000
:1014A00086E008C064E18FE005C067E185E102C025
:1014B00062E289E10E94142731CF83E20E944F1239
:1014C0002DCF2A960FB6F894DEBF0FBECDBFDF91A9
:1014D000CF911F910F91FF90EF90DF90CF90BF9031
:1014E000AF909F908F900895CF92DF92EF92FF92EE
:1014F0006C01EE24FF24C114D104E104F10421F0B5
:10150000C701B60120E101C020E0C72ED82EE92E88
:10151000FF24C114D104E104F10419F0285FC701CC
:10152000B6016B017C0154E0F694E794D794C7941C
:101530005A95D1F7C114D104E104F10419F02C5FDC
:10154000C701B6016B017C0142E0F694E794D794A1
:10155000C7944A95D1F7C114D104E104F10419F0FC
:101560002E5FC701B601DC01CB01B695A795979513
:101570008795892B8A2B8B2B09F02F5F822FFF9069
:10158000EF90DF90CF900895CF93DF93CDB7DEB784
:1015900064970FB6F894DEBF0FBECDBF84B7877FC8
:1015A00084BF0FB6F894A8958091600088618093FD
:1015B0006000109260000FBE90E080E80FB6F894D3
:1015C00080936100909361000FBE85B7806885BFEE
:1015D00085B7806885BF83EB96E190935302809333
:1015E00052020E94AA200E94C9208091E2008460D9
:1015F0008093E2007894809152038823A1F01091A7
:10160000E9001F709091EC00892F817090FD80E8B7
:10161000182B1092E9008091E80083FD0E94991D2B
:101620001F701093E90082E084BD93E095BD9AEFAE
:1016300097BD80936E0007ED11E07CEDE72E71E021
:10164000F72ED8018D918D018F3F11F00E94F81671
:10165000E016F106B1F70CED11E068EEE62E61E060
:10166000F62EF80181918F018F3F11F00E94F8163C
:10167000E016F106B1F78AE0E2E6F2E0DF01082FBA
:101680001D920A95E9F7E5E5F2E0DF011D928A95E2
:10169000E9F70E94BF2590937F0280937E020E940B
:1016A000BF2590937D0280937C0280E090E00E94B1
:1016B0001E2C893E9E4F11F00E94321B82E090E06A
:1016C0000E94102C80936C020E94211B9093530463
:1016D0008093520483E090E00E94102C682F70E009
:1016E00080E090E00E94232A0E94C72B80915F0235
:1016F000811136C080E090E00E941E2C893E9E4FF2
:1017000021F00E94321B0E94781088E090E00E9435
:10171000182C60933C0470933D0480933E04909396
:101720003F046E7F71F40E94781088E090E00E9480
:10173000182C60933C0470933D0480933E04909376
:101740003F040E9431101092A40280913C0480FF5B
:1017500004C060E086950E94141281E080935F02CD
:1017600028EF31E0AAEFB1E041E050E011E0AC3FFA
:10177000B10769F18D91E82FE295EF70F0E061A17A
:101780008F708A0102C0000F111F8A95E2F7C8010D
:10179000902F9095962391A392A1892B82A3F90172
:1017A00081919F01E82FE295EF70F0E061A18F70C9
:1017B0008A0102C0000F111F8A95E2F7C801902F1D
:1017C0009095962391A392A1892B82A3CFCF8FE8E6
:1017D00091E00197F1F700C0000089B18695817012
:1017E000489902C090E001C092E0892B8093840266
:1017F0008FB186958170789902C090E001C092E027
:10180000892B8093850288E991E090934A04809324
:10181000490458E1652E712C80915203853009F0FE
:1018200077C0FF24F39400E112E1809152038530E8
:1018300009F059C080915203843009F440C00E94DD
:10184000772B1092A40280916102811116C0F09250
:10185000610280913C04982F9170909360028E7F7A
:1018600080933C049FEFA0E7B2E09150A040B040CD
:10187000E1F700C000000E94EA0F10924D04E0E47E
:101880000FB6F894A895609260000FBEE0936000D8
:1018900083B7817F846083BF83B7816083BF78947F
:1018A000889583B78E7F83BF0FB6F894A8958091F3
:1018B0006000886180936000109260000FBE80918C
:1018C0005103882309F4B1CF0E940F17E2E6F2E03A
:1018D00081919191892B09F0F6C22CE632E02E1706
:1018E0003F07B1F7A2CF0E942D2A0E947D261092B9
:1018F000610280916002882349F080913C048160FC
:1019000080933C0460E086950E9414120E94D40FDC
:101910000E940F17882359F08FB7F89440914E0416
:1019200050914F0460915004709151048FBFA2E612
:10193000B2E0EDE6F2E000E010E0702F2D913D9175
:101940008191919182279327009779F160E0EE24AD
:10195000E394F12CAC014E215F21452B09F16F83FB
:1019600078872E213F2181E0232B09F480E08987AD
:101970000E94BF258160782F9B878A874F81588579
:1019800069858B850E94DC02000F111FF801E35965
:10199000FD4F80819181E826F926F182E0821AC00C
:1019A0006F5FEE0CFF1C6C30A9F60F5F1F4F053008
:1019B000110519F68FEF8C878D871E860E94BF2533
:1019C0008160782F988B8F874C855D856E8588899F
:1019D0000E94DC028091A402882309F493C08091C4
:1019E000A302E0913C04E695E81BE0939F0282305D
:1019F00059F4F0E0EA51FF4FE4910E2F10E091E925
:101A0000E92E94E2F92E59C0863059F4F0E0ED51F8
:101A1000FF4FE4910E2F10E081E8E82E84E2F82ECB
:101A20004CC0893061F4E695F0E0E052FF4FE4915C
:101A30000E2F10E0B7E1EB2EB4E2FB2E3EC08F304C
:101A400061F4E695F0E0E352FF4FE4910E2F10E0D1
:101A5000AAEAEA2EA3E2FA2E30C0853159F4F0E06A
:101A6000E652FF4FE4910E2F10E0FCE5EF2EF3E27B
:101A7000FF2E23C08831A1F0833249F4E8EDF0E075
:101A800005911491E1E4EE2EE4E2FE2E16C08432BC
:101A900071F404EF11E079E9E72E72E2F72E0DC040
:101AA00008E210E063EDE62E62E2F62E06C000EDDD
:101AB00017E055E0E52E52E2F52E8091A002882332
:101AC00061F01092A0020E94BF2590939E02809325
:101AD0009D021092A2021092A1020E94BF25E091E5
:101AE0009D02F0919E028E1B9F0B8F3F9F4750F4EB
:101AF0000E0F1F1F10939E0200939D028DE992E02E
:101B0000F701099504E812E01C8B0B8B82E8C82EC4
:101B100082E0D82E90E8E92E92E0F92E08EF11E04D
:101B20001A8B098B2AEF222E21E0322E34E8432E25
:101B300032E0532E912CB12C48E7A42E88248394B4
:101B4000D2018D912D01E82FEE0FEE0FD1012D91D5
:101B50001D01A22FA295AF70B0E090968C9190E0FD
:101B60002F7002C0959587952A95E2F79C01217008
:101B70003327A989BA898D91BA8BA98BA82FA295F1
:101B8000AF70B0E090964C9150E08F7002C05595C8
:101B900047958A95E2F7CA018170992740FF02C0F4
:101BA00082E090E0822B932B8E2BEB89FC89819332
:101BB000FC8BEB8B8F70E82FF0E0E851FE4F9081AB
:101BC000D6018C91890F8C938430B4F1F701808118
:101BD0008F5F80830E94BF2590937F0280937E0257
:101BE0000E94BF2590937D0280937C0260917802D1
:101BF0007091790280917A0290917B020E94740A1E
:101C0000FFEFF093770290E0A89E8001A99E100D4F
:101C10001124B11003C0025A1E4F02C0065B1E4FB2
:101C2000F801859194910E94B32AF80185919491CD
:101C30000E94532A21E001C020E0D6018C918D3F03
:101C4000A4F5F7018081815080830E94BF25909385
:101C50007F0280937E020E94BF2590937D02809335
:101C60007C02609178027091790280917A02909161
:101C70007B020E94740A8092770290E0A89E800105
:101C8000A99E100D1124B11003C0005A1E4F02C0AE
:101C9000045B1E4FF801859194910E94B32AF801CC
:101CA000859194910E94532A21E0D6018C91082EAF
:101CB000000C990B64E070E00E943F2EF6018193C6
:101CC0006F01922AB394FFEFEF1AFF0A02E0B012FD
:101CD00037CF992059F08FB7F89440914E04509126
:101CE0004F0460915004709151048FBF86E0E7E982
:101CF000F2E0DE01119601900D928A95E1F7E090F5
:101D00009902F0909A0200919B0210919C0210920D
:101D1000990210929A0210929B0210929C02E1107A
:101D200003C0FF2009F451C0809195029091960262
:101D30000E94B0259C0190919102992309F4D9C089
:101D40002531310508F441C09F3F19F09F5F909302
:101D50009102EE2061F00E9428131E1414F09FEFF0
:101D600001C091E0899F802D112480939902FF206A
:101D700061F00E9428131F1414F09FEF01C091E03E
:101D8000899F802D112480939A02309199023323E8
:101D9000E1F020919A022223C1F045EB3403C00107
:101DA0001124992319F09093990203C081E0809344
:101DB000990235EB2303C0011124992319F0909364
:101DC0009A0203C081E080939A02011103C011239B
:101DD00009F451C080919302909194020E94B02521
:101DE0009C0190919002992309F488C02135310516
:101DF00008F441C09F3F19F09F5F90939002002329
:101E000061F00E940613101614F09FEF01C091E0DC
:101E1000899F802D112480939B02112361F00E94E1
:101E20000613111614F09FEF01C091E0899F802DD9
:101E3000112480939C0230919B023323E1F0209186
:101E40009C022223C1F045EB3403C00111249923E5
:101E500019F090939B0203C081E080939B0235EBC5
:101E60002303C0011124992319F090939C0203C00D
:101E700081E080939C028091990281110BC0809136
:101E80009A02811107C080919B02811103C0809149
:101E90009C0281110E946512EB82FC820D831E83DD
:101EA00086E0FE013196A7E9B2E001900D928A9595
:101EB000E1F70E947D2690918602891709F4ACCC47
:101EC00080938602A9CC09BD19BD09B400FEFDCFDF
:101ED0008091D8008F7D8093D8008091E00082604F
:101EE0008093E0008091E00081FDFCCF0E942D2ACC
:101EF0009CCC2B30310508F029CF67CF2B30310532
:101F000008F07ACFB8CFCF92DF92EF92FF926B01B9
:101F10007C0120E030E0A9010E94582C811106C00C
:101F2000809180008F738093800039C08091800001
:101F3000806880938000C0928802D0928902E092EB
:101F40008A02F0928B0220E030E040E051E4C701C9
:101F5000B6010E94B02D9B01AC0160E074E284E701
:101F60009BE40E945D2C6B017C010E94CF2C70933E
:101F700087006093860020E030E048E452E4C70127
:101F8000B6010E94B02D20E030E048EC52E40E94FF
:101F90005D2C0E94CF2C7093890060938800FF9085
:101FA000EF90DF90CF90089560913C04669570E0CB
:101FB0004BE050E085EA91E00E94B82E892B19F49D
:101FC00081E08093A4020E94BF2590939E0280939B
:101FD0009D02089580913C0480FF0AC0859A81B3D8
:101FE0008F7D91B390622FB7F894EFEAF3E00BC0C6
:101FF000EFEAF3E0118210821282339634E0EC3380
:10200000F307C1F7EBCF34E0EC33F30789F03191FC
:1020100048E091BB000000C037FF81BB330F0000D8
:1020200000C000C000C081BB00C04A9591F7EBCF53
:102030002FBF8FE594E00197F1F700C000000895ED
:1020400090913C0490FF0CC0EFEAF3E08183608341
:102050004283339694E0EC33F907C1F70C94EA0F0E
:10206000089580913C04282F269530E021153105F4
:1020700019F48170826005C02532310524F0817029
:10208000886480933C040895CF92DF92EF92FF9290
:102090006B017C010E943110B701A60188E090E03D
:1020A000FF90EF90DF90CF900C94362C80914004FD
:1020B000882319F081508093400460913C04709112
:1020C0003D0480913E0490913F040C944410809113
:1020D0004004833018F48F5F8093400460913C0487
:1020E00070913D0480913E0490913F040C94441003
:1020F000ECE3F4E083E0808311828FEF82838383BB
:10210000148260817181828193810C944410AF921A
:10211000BF92CF92DF92EF92FF920F931F93CF93D4
:10212000DF93E82EF62EE901E42FF0E0611106C0FE
:10213000E652FE4FE4914E2F2E2F71C0062F10E075
:10214000E652FE4F4491F42FC42ED12C26E0829FFC
:10215000C00111242FEF30E0B9010E942B2E5BEA61
:102160005603C001579F900D11248E0D911D8E0DA9
:10217000911D582F550F580FD901A01BB10BAC9DC5
:10218000C001AD9D900DBC9D900D1124E92FF59ED1
:10219000D0011124AB2FBB277901EA1AFB0AEC9C72
:1021A000D001ED9CB00DFC9CB00D11245901A51A75
:1021B000B108A09E7001A19EF00CB09EF00C1124FD
:1021C000EF2CFF242E193F092C9D80012D9D100D11
:1021D0003C9D100D1124212F6230710591F048F4BF
:1021E00061157105E1F061307105B9F4242F4B2FB1
:1021F00016C06430710569F040F06630710579F001
:102200000CC0242F492FE12F0AC0492FEF2F2B2F6D
:1022100006C0292FE42F412F02C0292FEB2F49831D
:102220002883EA83DF91CF911F910F91FF90EF9068
:10223000DF90CF90BF90AF900895CF93DF9300D001
:102240001F92CDB7DEB790913C0490FF0AC09E016B
:102250002F5F3F4F0E9487104B8169818A810E94C6
:1022600020100F900F900F90DF91CF9108955F9203
:102270006F927F928F929F92AF92BF92CF92DF9296
:10228000EF92FF920F931F93CF93DF9300D01F9293
:10229000CDB7DEB7182F762E042F622E90913C0416
:1022A00090FF6DC0E92FE695AE2FB0E0A450BE4F71
:1022B0008C918093A3029E7F923061F49E012F5FE8
:1022C0003F4F812F0E9487104B8169818A810E9434
:1022D000201043C0823019F400913F043EC0863084
:1022E00019F410913D0439C08930D9F38931A9F529
:1022F000E9518E2F8170582EE695F0E0E652FD4FA1
:10230000A590B4908FEAC82E83E0D82EE12CF12C52
:10231000BB249FE2892E912CAE9CC001AF9C900DF6
:10232000BE9C900D1124B4010E942B2E812F5110C0
:1023300002C0860F01C0861B9601402F672D0E94A8
:1023400087108FEFE81AF80A83E0C80ED11C8FE2DD
:10235000E816F10409F70E94EA0F10933D04709209
:102360003E0400933F04662051F060913C0470915C
:102370003D0480913E0490913F040E9444100F90D0
:102380000F900F90DF91CF911F910F91FF90EF90E1
:10239000DF90CF90BF90AF909F908F907F906F9085
:1023A0005F900895ECE3F4E0438128E0421B08F4D9
:1023B00040E021E0628181810C943711ECE3F4E08C
:1023C000438128E0420F08F44FEF21E062818181D0
:1023D0000C943711ECE3F4E0628128E0621B08F40E
:1023E00060E021E0438181810C943711ECE3F4E05B
:1023F000628128E0620F08F46FEF21E04381818160
:102400000C943711ECE3F4E0818121E04381628197
:1024100088500C943711ECE3F4E0818121E0438192
:102420006281885F0C94371190913C0490FF36C014
:102430009170811102C0926006C0853210F09864DC
:1024400002C0880F982B90933C04662351F0609152
:102450003C0470913D0480913E0490913F040E94A1
:10246000441060913C04669570E04BE050E085EAD2
:1024700091E00E94B82E892B19F01092A40202C09C
:102480000E94D40F81E08093A00220E040913F049D
:1024900060913E0480913D040C943711089561E0F1
:1024A0000C94141280913C048695815009F484E2C6
:1024B00061E00C94141280913C0486958F5F853204
:1024C00008F081E061E00C9414120E94BF25209175
:1024D0009902211104C020919A02222321F09093A5
:1024E00096028093950220919B02211104C02091B5
:1024F0009C02222321F09093940280939302E09116
:102500004904F0914A04309749F082E080939702A1
:102510000480F581E02D87E992E0099408958D3ECD
:1025200039F490919A0297FF35C010929A0259C0DF
:102530008E3E29F490919A021916BCF32BC090910B
:1025400099028F3E29F497FF25C01092990249C045
:10255000803F19F41916CCF31DC090919B02893F5E
:1025600029F41916BCF410929B023BC08A3F19F45F
:1025700097FF10C0F8CF8B3F39F490919C0297FFE2
:1025800009C010929C022DC08C3F21F490919C02B6
:102590001916BCF39FE0980F983080F421E030E0EA
:1025A000A90102C0440F551F9A95E2F7CA01809510
:1025B0009091980289238093980213C08D3F21F453
:1025C000809192028E7F0BC08E3F21F48091920207
:1025D0008D7F05C08F3F29F4809192028B7F80937D
:1025E000920280919902811106C080919A02811114
:1025F00002C01092910280919B02811106C08091CD
:102600009C02811102C01092900208958091920262
:1026100080FD16C081FD16C082FD18C08091900219
:10262000882391F0883290F428E0829FC001112421
:1026300068E270E00E943F2E862F672B29F007C0CA
:1026400082E0089584E0089581E0089588E0089587
:102650008091920280FD14C081FD14C082FD16C0DD
:1026600080919102882381F08E3180F420E5829F51
:10267000C00111246EE170E00E943F2E862F089564
:1026800084E1089588E2089588E0089580E508953A
:102690008D3E21F40E942813819504C08E3E29F4BA
:1026A0000E94281380939A0208958F3E21F40E947D
:1026B0002813819504C0803F29F40E942813809339
:1026C00099020895893F19F40E94061305C08A3FB4
:1026D00031F40E940613819580939B0208958B3FED
:1026E00021F40E940613819504C08C3F29F40E94B6
:1026F000061380939C0208959FE0980F983078F419
:1027000021E030E0A90102C0440F551F9A95E2F77D
:10271000CA0190919802892B8093980208958D3F69
:1027200021F48091920281600BC08E3F21F4809150
:102730009202826005C08F3F29F4809192028460EA
:10274000809392020895EFE6F0E080818D7F808390
:10275000E0E8F0E080818F73808308957F928F920C
:102760009F92AF92BF92CF92DF92EF92FF920F9320
:102770001F93CF93DF934B015C016A0180916B0340
:1027800080FFAEC080916A03811102C00E94C72BF6
:1027900020E030E0A901C501B4010E94582C87FF58
:1027A00004C0B7FAB094B7F8B0947090AE03072D98
:1027B00010E0E801219743E0000F111F4A95E1F76F
:1027C000E12CF12CCF3FFFEFDF07D9F128E0E21A2F
:1027D000F108F801EE0DFF1DE259FC4F2281338113
:1027E00044815581C501B4010E94582C811127C034
:1027F0008E0133E0000F111F3A95E1F702591C4F8B
:102800008091AE0390E00197C817D9070CF068C01B
:10281000219688E0F8013896D80101900D928A95AA
:10282000E1F70E94BF25F801918780878286938611
:10283000A486B586D786C686085F1F4FE1CF21974D
:10284000C1CF81E0870D893020F58093AE0381E010
:102850008093870280936903C091AE03D0E02197F3
:102860000E94BF25FE0123E0EE0FFF1F2A95E1F72E
:10287000E259FC4F9183808382829382A482B58245
:10288000D782C6820E94BF258091A401882341F18E
:1028900013C088E08093AE038EE693E028E0FC014D
:1028A0003896DC0101900D922A95E1F7089623E015
:1028B000863A920799F7CBCF80916F008260809320
:1028C0006F00809180008068809380008091690310
:1028D000882321F00E94C41C0E94830F1092A4013F
:1028E000DF91CF911F910F91FF90EF90DF90CF90EC
:1028F000BF90AF909F908F907F9008951F920F92FE
:102900000FB60F9211242F923F924F925F926F92C7
:102910007F928F929F92AF92BF92CF92DF92EF926F
:10292000FF920F931F932F933F934F935F936F9358
:102930007F938F939F93AF93BF93CF93DF93EF9347
:10294000FF9380918C0290918D02A0918E02B091A4
:102950008F020196A11DB11D80938C0290938D0270
:10296000A0938E02B0938F0260918C0270918D02C1
:1029700080918E0290918F020E94FE2C6B017C014F
:1029800020E030E040E85CE36091880270918902C9
:1029900080918A0290918B020E94B02D9B01AC0124
:1029A000C701B6010E94582C87FDBAC110928C0253
:1029B00010928D0210928E0210928F028091690304
:1029C000811105C0C0916803CC2309F498C10E940D
:1029D000BF25EC0180916803811102C0312CE4C055
:1029E00080915E0390915F030E94B02520915C036B
:1029F00030915D038217930788F380915E03909175
:102A00005F030E94B02520915C0330915D037C013F
:102A1000E21AF30AD0935F03C0935E030091600350
:102A200010916103C8010196909361038093600344
:102A30000E94BF25A0906303B0906403809160035F
:102A4000909161038A159B0560F0C0916203CC23CD
:102A500029F0109261031092600303C00E94772B4B
:102A60004EC180916703C0916003D0916103C09013
:102A70006503D0906603811131C0F80163E0EE0F69
:102A8000FF1F6A95E1F7EC0DFD1DDE0173E0AA0F53
:102A9000BB1F7A95E1F7AC0DBD1D2D913D914D9178
:102AA0005C9160817181828193810E94582C811197
:102AB00015C081E0809367034FE050E060E070E074
:102AC000CB010E94AE1310936103009360038FE06B
:102AD00090E090935D0380935C0364C01092670361
:102AE0008E0143E0000F111F4A95E1F70C0D1D1DEB
:102AF000F80164817581868197810E94CF2C9B01AA
:102B0000A0E6BAEE0E94832E20E03EE140E050E0D5
:102B10000E94532EF1E0AF1AB108412C5EE1552E10
:102B2000612C712C2E153F0550F0D0936103C0939A
:102B30006003E216F306E0F0C1E0D0E01CC0085FDD
:102B40001F4FCA15DB0588F7E21AF30A2196F80130
:102B500064817581868197810E94CF2C9B01A0E6BC
:102B6000BAEE0E94832EA30192010E94532EDACF67
:102B7000E901CE19DF09809160039091610333E090
:102B8000880F991F3A95E1F7F601E80FF91F608168
:102B9000718182819381AE010E94AE13D0935D0357
:102BA000C0935C033324339480916903882309F430
:102BB0009EC080916C03882311F0332433940EE679
:102BC00013E0812C912C412C512C20E8622E2FEB0C
:102BD000722E222423948091AE0390E088169906E9
:102BE0000CF085C0F8018681978101978E3F9F4F39
:102BF00008F077C0F801808191810E94B025F8012A
:102C0000268137818217930708F46BC0C280D38076
:102C1000E480F58020E030E0A901C701B6010E9400
:102C2000582C87FF04C0F7FAF094F7F8F0948091DD
:102C30006903882309F455C080916A03811102C099
:102C40000E94C72B9EE6A92E93E0B92EC7E0D0E0E4
:102C5000A7019601F50162AD73AD84AD95AD0E94FB
:102C6000582C811126C083E0CC0FDD1F8A95E1F737
:102C7000C259DC4F198218824A825B826C827D8243
:102C80001F821E8286EA93E08C179D07D9F088E0A8
:102C9000FE013896DE0101900D928A95E1F71986C2
:102CA00018864A865B866C867D861F861E862896D9
:102CB000E9CF219798E0A91AB108CF3FEFEFDE07DF
:102CC00039F60FC0209287028091AE038150809325
:102CD000AE03811106C00E94A3132092A40110929A
:102CE0006903FFEF8F1A9F0A085F1F4F74CFC091CF
:102CF0008702CC2319F01092870201C0C32D809166
:102D00006903811107C080916803811103C00E948B
:102D1000A31306C0CC2321F00E94C41C0E94830F81
:102D2000FF91EF91DF91CF91BF91AF919F918F91E3
:102D30007F916F915F914F913F912F911F910F91D3
:102D4000FF90EF90DF90CF90BF90AF909F908F90CB
:102D50007F906F905F904F903F902F900F900FBE9D
:102D60000F901F90189580E008959091520492FF63
:102D70000DC0282F2871283019F4877F846006C081
:102D8000282F2471243011F48B7F886093FF0DC0AD
:102D9000282F2871283119F4877E846106C0282FD6
:102DA0002471243111F48B7E88612091530420FF1B
:102DB0000DC0382F3871383019F4877F816006C014
:102DC000382F3171313011F48E7F886021FF0DC0B2
:102DD000282F2871283119F4877E816106C0282F99
:102DE0002171213111F48E7E886194FD877E0895D2
:102DF000F894E82FE295EF70F0E031A1282F2F70C2
:102E000081E090E001C0880F2A95EAF7982F90950D
:102E1000932391A392A1892B82A3789408956F9212
:102E20007F928F929F92AF92BF92CF92DF92EF925A
:102E3000FF920F931F93CF93DF93CDB7DEB72A97FF
:102E40000FB6F894DEBF0FBECDBFAE014F5F5F4F30
:102E50007A018AE0FA0111928A95E9F707ED11E00B
:102E60006A019CED692E91E0792E88248394912C3F
:102E7000F80180818F3F09F447C0F894E82FE2956C
:102E8000EF70F0E021A18F70A40102C0440F551F24
:102E90008A95E2F7CA01922F982B91A392A180956F
:102EA000892382A3789400C0ECEDF1E021E030E0CA
:102EB000A12CB12C41914F3F89F0A42FA295AF7066
:102EC000B0E090968C9190E04F7002C095958795F8
:102ED0004A95E2F780FD02C0C90102C080E090E09F
:102EE000A82AB92A220F331F51E0E83EF50711F74F
:102EF000F80180818F3F11F00E94F816F0EAFA95F0
:102F0000F1F7F601B182A0820F5F1F4FF2E0CF0E02
:102F1000D11C6016710609F0ABCF4AE050E0B70152
:102F200085E592E00E94C52E01E0009709F400E0DB
:102F3000892B89F08AE0F701A5E5B2E001900D92B6
:102F40008A95E1F781E0809327030E94BF25909343
:102F500026038093250380912703882391F1809194
:102F60002503909126030E94B025059750F180918A
:102F70005502909156029093630280936202809171
:102F80005702909158029093650280936402809159
:102F9000590290915A029093670280936602809141
:102FA0005B0290915C029093690280936802809129
:102FB0005D0290915E0290936B0280936A02109280
:102FC0002703609178027091790280917A02909142
:102FD0007B020E94740A182F80917702882309F4DB
:102FE00074C080917E0290917F020E94B025893743
:102FF000954038F0109277028091B1010E944F12F3
:1030000064C080917C0290917D020E94B0258D3B2E
:10301000924058F040E060E080E00E9420100E9462
:10302000BF2590937D0280937C0280917C029091D9
:103030007D020E94B0258135910558F0809177027C
:10304000813011F443E101C040E160E880E80E9472
:10305000AF1C80917C0290917D020E94B025853B3F
:10306000910558F080917702813011F448E001C059
:1030700043E060EA80EA0E94AF1C80917C0290915C
:103080007D020E94B0258931914058F080917702ED
:10309000813011F449E001C042E060EC80EC0E9414
:1030A000AF1C80917C0290917D020E94B0258139F5
:1030B000914058F080917702813011F44AE001C0CC
:1030C00041E060EE80EE0E94AF1C80912C03181747
:1030D00029F081E08093B00110932C038091B0011E
:1030E000882309F4FEC0111105C08091B1010E942E
:1030F0004F12F5C081E00E944F12809128039091F9
:10310000290340E050E0FCE31F9FB0011124A0EC34
:1031100020E830E4B5E04033510509F4D6C0CA01D7
:103120004A32510508F00197FB01E40FF51FEE0F3D
:10313000FF1FE651FF4FE590F490E1E0EE16F10439
:1031400059F4FC01EE0FFF1FE80FF91FE155FC4F8A
:10315000B183B083B283B6C0EF2851F4FC01EE0F07
:10316000FF1FE80FF91FE155FC4F118210820BC0C1
:10317000113059F4FC01EE0FFF1FE80FF91FE15564
:10318000FC4F2183308312829DC0123051F4FC0128
:10319000EE0FFF1FE80FF91FE155FC4F118230833E
:1031A00090C0133049F4FC01EE0FFF1FE80FF91F28
:1031B000E155FC4F318323C0143051F4FC01EE0F74
:1031C000FF1FE80FF91FE155FC4F1182208330C02B
:1031D000153011F0163049F4FC01EE0FFF1FE80F17
:1031E000F91FE155FC4F21835FC0173051F4FC01FA
:1031F000EE0FFF1FE80FF91FE155FC4F21832083DD
:10320000C2CF183051F4FC01EE0FFF1FE80FF91F79
:10321000E155FC4F1182208354C0193059F4FC0150
:10322000EE0FFF1FE80FF91FE155FC4F2183A0832C
:10323000328348C01A3049F4FC01EE0FFF1FE80F3B
:10324000F91FE155FC4F31833BC01B3051F4FC01A9
:10325000EE0FFF1FE80FF91FE155FC4F218330836C
:103260000BC01C3059F4FC01EE0FFF1FE80FF91FD3
:10327000E155FC4F31832083A28324C01D3051F4DB
:10328000FC01EE0FFF1FE80FF91FE155FC4F2183F2
:10329000A08379CF1E3051F4FC01EE0FFF1FE80F21
:1032A000F91FE155FC4FA18310820BC01F3051F470
:1032B000FC01EE0FFF1FE80FF91FE155FC4F1182D3
:1032C000A08322834F5F5F4F26CF90932903809383
:1032D000280350932B0340932A030E94EA0F109275
:1032E000B001802F2A960FB6F894DEBF0FBECDBF77
:1032F000DF91CF911F910F91FF90EF90DF90CF90D2
:10330000BF90AF909F908F907F906F900895CF93D4
:10331000DF938238910569F1B0F48133910509F4A6
:103320006FC048F48932910509F465C08A3291056D
:1033300009F46BC08AC08533910509F457C08933FD
:103340009105B9F082C0833E910571F138F4803E59
:103350009105B1F0823E910511F177C0863E91054D
:10336000B9F1873E9105C9F1843E910509F06DC020
:1033700024C02091520420FD53C021FD51C065C0DE
:103380008091520480FD46C08091530480FF48C064
:103390008091520484FD50C183EE90E04FC1809132
:1033A000520482FF3AC0F4CF8091520482FD35C0AE
:1033B0008091530480FD34C0EBCF8091530481FF92
:1033C00035C08091520484FD37C187EE90E036C14C
:1033D0008091520483FF27C0F4CF8091520483FD73
:1033E00022C08091530481FD21C0EBCF8091520413
:1033F00085FD1FC021C08091520485FD1DC019C0EC
:103400008091520486FD1BC01DC08091520486FD30
:1034100019C015C089E390E011C182EE90E00EC1A1
:1034200080EE90E00BC186EE90E008C184EE90E063
:1034300005C189E290E002C185E390E0FFC08AE225
:1034400090E0FCC081E390E0F9C0811531E593077D
:1034500008F069C0811540E59407F0F09C0174E024
:10346000369527957A95E1F7922F9370482F437000
:1034700021E030E002C0220F331F4A95E2F73C689A
:10348000392B982F9F709695969540E2949FC00196
:103490001124822B932BD2C0883E910568F5803E83
:1034A000910508F0CBC0883A9105B8F4853A9105AA
:1034B00048F0855AE82FF0E0EF5DFD4F808190E005
:1034C0009064BCC08130910509F4B3C008F4B4C065
:1034D0008430910508F4B0C0B1C08F3B910508F06D
:1034E000ABC0885AE82FF0E0EE0FFF1FEC5DFD4FF8
:1034F000808191819464A2C0811520E2920758F4E2
:10350000811531E0930708F099C08D3E910508F4CC
:1035100093C0906593C0811540E4940708F48CC073
:103520009F70906A8BC0811525E5920708F042C014
:10353000811534E5930728F0982F8827846F906AC7
:103540007DC0811543E59407B0F09C0123703327BB
:1035500041E050E002C0440F551F2A95E2F7282FA2
:103560002695269580E2289F90011124CA01822B7E
:10357000932B9A6863C0811522E5920728F4982F4F
:103580008827816F906A5AC09C012370332741E0DD
:1035900050E002C0440F551F2A95E2F7282F2695C8
:1035A000269580E2289F90011124CA01822B932B3B
:1035B0009C6844C0EC01811539E59307A8F4811596
:1035C000984528F09C2F8827806F906A37C0C115D6
:1035D00086E5D80788F58C2F0E94B5168F7190E08C
:1035E000982F882790622AC081152AE5920790F4C7
:1035F0008C2F8F700E94B51694E0D695C7959A953A
:10360000E1F7CF70D0E0DC2FCC27D0699E01282BCA
:10361000C90114C090568115904270F48D2F8F719E
:103620000E94B516282F2F71CE0199279062922BF8
:1036300005C081E090E002C080E090E0DF91CF9192
:103640000895CF9384E090E00E94102CC82F82E26E
:1036500090E00E94102C2C2F30E0A901582BCA01B9
:10366000CF91089569EE7EEF80E090E00E94422CB9
:1036700060E082E090E00E94242C60E083E090E033
:103680000E94242C109221031092220310922303F3
:103690001092240360E084E090E00E94242C60E01B
:1036A00082E290E00E94242C60E085E090E00E949D
:1036B000242C60E086E090E00E94242C6FEF87E0ED
:1036C00090E00E94242C40E050E0BA0188E090E0B5
:1036D0000E94362C60E08DE090E00E94242C40E0B7
:1036E00050E0BA0188E190E00E94362C60E087E16A
:1036F00090E00E94242C40E050E0BA018CE190E080
:103700000E94362C60E070E080E290E00E94422C43
:1037100040E050E0BA0188E190E00E94362C40E0A1
:1037200050E0BA018FE090E00E94362C40E050E07B
:10373000BA0183E190E00C94362C80912003811132
:10374000109220030895809590911F038923809300
:103750001F03089590911F0380911E03982B90934F
:10376000A502809120038823D9F0892B8093A5029C
:103770008091B301882331F08091520487FF02C009
:103780008EE101C086E0E7EAF2E090E0815028F0A7
:1037900021912223D9F39F5FF9CF91110E949D1BA4
:1037A00040E250E06EEF72E085EA92E00E94C52EA2
:1037B000892B21F180E2E5EAF2E0AEEFB2E0019080
:1037C0000D928A95E1F7E0914904F0914A0430970F
:1037D000A9F08091B301882359F08091520487FFAA
:1037E00007C08091A5028093A60286E08093A5027F
:1037F0000280F381E02D85EA92E0099408952091FA
:10380000FD02809582238093FD02982F977099F492
:1038100030E0482F082E000C550B2417350759F0BF
:103820009091530492FD07C08595859585950E94DA
:10383000DD291092FD020895CF93C0915304C2FB7D
:10384000992790F9981799F080FBC2F9C093530417
:103850006091520484E090E00E94242C6C2F82E25C
:1038600090E00E94242C82E0CF910C94FF1BCF911A
:1038700008958091FC029091CB02891719F08F5F17
:103880008770FBCF08950F931F93CF93DF938091A1
:10389000CA0282958F7009F05DC08091C7028823AB
:1038A00009F458C08091FC021091CB026091C502CE
:1038B0007091C602C091C802D091C90291E06F3FD9
:1038C00009F090E0292F06E0811709F443C0209702
:1038D00021F07F3F21F030E003C031E001C0322F02
:1038E00090E030FD34C0089FF001099FF00D1124D5
:1038F000DF01A453BD4F11963C911197371327C098
:103900003C91361324C012963C91129731111FC07E
:1039100013964D915C9114974C1B5D0B483C5105DF
:10392000B0F48091CA028F7080618093CA02EF5216
:10393000FD4F80818F708061808385EC92E00E94D2
:103940008403DF91CF911F910F910C94391C019644
:103950008770BACFDF91CF911F910F910895909109
:103960003C0490FF10C04F3270F450E0FA01EE0FAB
:10397000FF1F4E0F5F1FFA01E155FC4F81836083EB
:1039800012820C94EA0F0895CF92DF92EF92FF9289
:10399000E091AE03EE23D9F0E15088E0E802F001B7
:1039A0001124E259FC4FC280D380E480F58020E0EE
:1039B00030E0A901C701B6010E94582C18163CF44A
:1039C00080916D03811106C010926C0303C0C12C5D
:1039D000D12C7601C701B601FF90EF90DF90CF9018
:1039E0000895CF92DF92EF92FF92CF93DF932091D1
:1039F0006B0320FD08C0DF91CF91FF90EF90DF9027
:103A0000CF900C94772B7B01EC0180916A0381119C
:103A100002C00E94C72B8091690381110E94772BFD
:103A200081E08093680310926703D0936603C0938C
:103A30006503F0926403E0926303109262031092B4
:103A40006103109260036C817D818E819F810E9451
:103A5000CF2C9B01A0E6BAEE0E94832EC12C2EE152
:103A6000D22EE12CF12CA70196010E94532E6881E1
:103A700079818A819B81A9010E94AE130E94BF2592
:103A800090935F0380935E0380916503909166033A
:103A9000E0916003F091610333E0EE0FFF1F3A9570
:103AA000E1F7E80FF91F64817581868197810E9493
:103AB000CF2C9B01A0E6BAEE0E94832EA7019601AF
:103AC0000E94532E30935D0320935C03DF91CF91CE
:103AD000FF90EF90DF90CF900895EF92FF920F93B9
:103AE0001F93CF93DF937C018B010E94A52481114A
:103AF00019C0E70101151105A1F08091E80085FDCD
:103B00000AC08091E8008E778093E8000E94A52487
:103B1000882381F307C089918093F1000150110936
:103B2000E9CF80E0DF91CF911F910F91FF90EF904F
:103B300008951F93CF93DF93CDB7DEB7AA970FB643
:103B4000F894DEBF0FBECDBFE4E5F3E08CE593E073
:103B50002091F10021938E179F07D1F78091550393
:103B6000833009F461C030F4813071F0823009F49F
:103B70009BC0B2C08A3009F487C08B3009F46CC096
:103B8000893009F0A9C020C080915403813A09F01E
:103B9000A3C08091E800877F8093E800809158035C
:103BA00090915903892B21F460E280E393E003C0F4
:103BB00060E080E090E070E00E942C258091E800B9
:103BC0008B778093E80088C080915403813209F09C
:103BD00083C08091580390915903029708F07CC0EC
:103BE0008091E800877F8093E8008091E80082FD63
:103BF00005C0809152038111F8CF6EC02091F3006F
:103C00008091F20090E0922B029731F48091F100C4
:103C1000813011F0863021F48091F10080932F03E0
:103C20008091E8008B7754C080915403813A09F069
:103C300053C08091580390915903892B09F04CC0CF
:103C40008091E800877F8093E8008091E80080FF02
:103C5000FCCF8091B30137C0809154038132E1F5EC
:103C60008091580390915903892BB1F58091E80018
:103C7000877F8093E8000E94D82480915603809328
:103C8000B3010E942D2A28C080915403813221F56E
:103C90008091E800877F8093E8000E94D82480917B
:103CA000570380932E0318C080915403813AA1F4E6
:103CB0008091E800877F8093E8008091E80080FF92
:103CC000FCCF80912E038093F1008091E8008E77E5
:103CD0008093E8000E94D8248091E80083FFCEC141
:103CE0008091540390915503492F50E04A3051057B
:103CF00008F0C4C1FA01EE59FF4F0C94752E8038BC
:103D000021F0823809F0BAC108C080915003909127
:103D10005103992389F082600FC0809158038F70FE
:103D2000873008F0ABC18093E9008091EB0085FB00
:103D3000882780F91092E9009091E800977F90938E
:103D4000E8008093F1001092F10065C1282F2D7FCB
:103D500009F094C1882319F0823061F08FC18091FD
:103D60005603813009F08AC1933009F080E08093D6
:103D700051032EC08091560381112AC080915803AF
:103D80008F702FEF280F263008F078C18093E9005C
:103D90002091EB0020FF1CC0933021F48091EB00B8
:103DA000806214C09091EB0090619093EB0021E051
:103DB00030E0A90102C0440F551F8A95E2F74093F5
:103DC000EA001092EA008091EB0088608093EB009B
:103DD0001092E9008091E800877F20C181114EC1D7
:103DE000109156031F778091E3008078812B809398
:103DF000E3008091E800877F8093E8000E94D82448
:103E00008091E80080FFFCCF8091E3008068809380
:103E1000E300111102C082E001C083E080935203ED
:103E20002DC18058823008F029C1809156039091AD
:103E300057038C3D53E0950779F583E08A838AE246
:103E400089834FB7F894DE01139620E03EE051E2FB
:103E5000E32FF0E050935700E49120FF03C0E29578
:103E6000EF703F5FEF708E2F90E0EA3010F0C79652
:103E700001C0C0968D939D932F5F243149F74FBFAA
:103E80008091E800877F8093E8006AE270E0CE01CD
:103E900001960E942C25AEC04091580350915903C1
:103EA000292F332723303105A9F068F4213031055B
:103EB00009F4F3C02230310509F0E0C08BE390E053
:103EC000E5EDF3E044C02132310521F12232310524
:103ED00071F1D4C0992781309105A1F058F0029773
:103EE00009F0CCC0E2E2F4E0E4918E2F90E0E2E24F
:103EF000F4E02AC0E0E4F4E0E4918E2F90E0E0E406
:103F0000F4E022C0E2E3F4E0E4918E2F90E0E2E3FB
:103F1000F4E01AC04115510509F4C4C041305105FF
:103F200009F0ACC089E090E0E0E0F4E010C0411599
:103F3000510509F4BCC04130510509F09FC086EB22
:103F400090E0EFEDF2E003C0009709F497C02091F4
:103F5000E800277F2093E80020915A0330915B030B
:103F60008217930708F49C0140E02115310589F17F
:103F700080915203882309F43DC08530D9F18091A6
:103F8000E80083FD37C08091E80082FD2FC080915A
:103F9000E80080FFEACF4091F3008091F20090E0CA
:103FA000942B2115310559F08830910540F4449146
:103FB0004093F1003196215031090196F2CF41E052
:103FC000089709F040E08091E8008E778093E80040
:103FD000CCCF4111CDCF0AC080915203882351F03C
:103FE000853041F08091E80083FD04C08091E800B5
:103FF00082FFF2CF8091E8008B778093E8003EC08B
:104000008038E1F58091E800877F8093E800809117
:1040100053038093F1008091E8008E778093E8004D
:104020000E94D8242BC0811129C080915603909101
:1040300057039927029714F58091E800877F8093B2
:10404000E80010915603109353030E94D8241111D5
:1040500006C08091E30087FD02C081E001C084E0DA
:104060008093520342E061EC81E00E94F72442E237
:1040700061EC82E00E94F724809152038091E80075
:1040800083FF1AC08091E800877F8093E8008091C9
:10409000EB0080628093EB000FC082E190E0E0E1F2
:1040A000F4E055CF89E090E0E7EEF3E050CF80E414
:1040B00090E0E5E9F3E04BCFAA960FB6F894DEBFA7
:1040C0000FBECDBFDF91CF911F9108951F920F9228
:1040D0000FB60F9211242F933F934F935F936F93DB
:1040E0007F938F939F93AF93BF93CF93DF93EF9380
:1040F000FF93C091E900CF708091EC00D82FD17070
:1041000080FDD0E81092E9008091F000877F8093D5
:10411000F00078940E94991D1092E9008091F000BF
:1041200088608093F000CD2BCF70C093E900FF91A1
:10413000EF91DF91CF91BF91AF919F918F917F913F
:104140006F915F914F913F912F910F900FBE0F9004
:104150001F901895E8EDF0E080818E7F80831092AB
:10416000E2001092DA001092E100A0EEB0E08C9133
:1041700081608C9380818F77808319BCA7EDB0E03C
:104180008C918E7F8C9380818F7E808310922D0303
:104190000895CF92DF92EF92FF920F931F93CF93E8
:1041A000DF93C8EDD0E088818F7E8883E7EDF0E073
:1041B00080818160808384E082BF81E080932D03D1
:1041C00088818E7F888302EE10E0F80110821092C1
:1041D000DA0081EEC82ED12CF601108288818F770B
:1041E000888388818068888388818F7D888319BCD3
:1041F00010925203109253031092510310925003E5
:1042000090EEE92EF12CF70180818B7F80838881ED
:104210008160888342E060E080E00E94F724F6013C
:1042200080818E7F8083F80180818160808380819E
:1042300088608083F70180818E7F808388818061A0
:104240008883DF91CF911F910F91FF90EF90DF90C6
:10425000CF9008951F920F920FB60F9211242F93B3
:104260003F934F935F936F937F938F939F93AF93FE
:10427000BF93EF93FF938091E10082FF09C080918B
:10428000E20082FF05C08091E1008B7F8093E10016
:104290008091DA0080FF2AC08091D80080FF26C07C
:1042A0008091DA008E7F8093DA008091D90080FFC0
:1042B00018C080E189BD82E189BD09B400FEFDCF4F
:1042C00081E08093520380912D0381110FC00E94E1
:1042D000AA200E94C9208091E20084608093E200BD
:1042E00005C019BC1092520310922D038091E10079
:1042F00080FF17C08091E20080FF13C08091E20030
:104300008E7F8093E2008091E20080618093E200E2
:104310008091D80080628093D80019BC85E080939A
:1043200052038091E10084FF30C08091E20084FF5D
:104330002CC080E189BD82E189BD09B400FEFDCFBA
:104340008091D8008F7D8093D8008091E1008F7E8E
:104350008093E1008091E2008F7E8093E200809163
:10436000E20081608093E20080915303882311F082
:1043700084E007C08091E30087FD02C081E001C0B6
:1043800083E080935203809152038091E10083FF88
:1043900027C08091E20083FF23C08091E100877FE6
:1043A0008093E10082E08093520310925303809146
:1043B000E1008E7F8093E1008091E2008E7F809308
:1043C000E2008091E20080618093E20042E060E0E0
:1043D00080E00E94F7248091F00088608093F000D4
:1043E000FF91EF91BF91AF919F918F917F916F91CD
:1043F0005F914F913F912F910F900FBE0F901F90A3
:104400001895089580912F0308950895809354047A
:10441000709356046093550480915203843001F5E3
:1044200082E08093E9008FEF9091E800815095FD44
:1044300006C095ED9A95F1F700008111F5CF8091B6
:10444000E80085FF0DC040E050E063E070E084E5E7
:1044500094E00E946D1D8091E8008E778093E800C3
:104460000895BC0184E00C940622BC0183E00C9406
:10447000062222E02093E9002FEF3091E80021503E
:1044800035FD06C035ED3A95F1F700002111F5CF65
:104490002091E80025FF0BC040E050E066E070E0AE
:1044A0000E946D1D8091E8008E778093E80008954A
:1044B000CF93DF932091B301222339F0209152044E
:1044C00027FF03C060E222E002C068E021E0209301
:1044D000E9002FEF3091E800215035FD06C035EDA1
:1044E0003A95F1F700002111F5CF2091E80025FF62
:1044F0001DC0EC018091B301811105C040E050E086
:1045000068E070E003C070E040E050E0CE010E943F
:104510006D1D8091E8008E778093E80080E2FE01B7
:10452000A0E3B3E001900D928A95E1F7DF91CF917E
:104530000895EF92FF920F931F93CF93DF938C0117
:10454000CFEAD3E0E12CF12CF8018481F7E1EF16FA
:10455000F1041CF4882339F002C0811104C09E01CB
:1045600040913F0402C09E0140E060913E04809172
:104570003D040E9487108FEFE81AF80A23969FE205
:10458000E916F10409F70E94EA0FF801848190E02E
:104590000196817099278483DF91CF911F910F91AC
:1045A000FF90EF9008958F929F92AF92BF92CF921B
:1045B000DF92EF92FF920F931F93CF93DF93EC0163
:1045C0004C81042F10E09801D8010E94832E9B019A
:1045D000AC010E94992E6B017C01E0E2F0E0E01B4F
:1045E000F10BA5E5B0E09B01AC010E94992E4B01B7
:1045F0005C019F01DF010E947B2E9B01AC010E94A8
:10460000A42E9B01AC012C0D3D1D4E1D5F1DC5014F
:10461000B4010E94532E822FF22E99E2921728F0B5
:1046200093E0299F900111240DC025E530E0281B5F
:104630003109C901880F991F280F391F37FF02C0A0
:104640002F5F3F4F35952795122F10959FEAC92E62
:1046500093E0D92E00E085E5E82EEF1801FD02C0B9
:104660008E2D01C08F2D9601412F60913E040E9436
:1046700087100F5F83E0C80ED11C0F3279F70E94BC
:10468000EA0F8C81811102C091E003C0803219F4DD
:104690009FEF9093B6019091B601890F8C83DF91C3
:1046A000CF911F910F91FF90EF90DF90CF90BF902F
:1046B000AF909F908F9008950F931F93CF93DF93A8
:1046C000CFEAD3E0FE01118210821282339684E099
:1046D000EC33F807C1F700E010E080914204082EA7
:1046E000000C990B0817190794F08091B501082E5A
:1046F000000C990B8017910754F09E0140913F04E4
:1047000060913E0480913D040E94871003C019828D
:1047100018821A820F5F1F4F23960C301105E9F69D
:104720000E94EA0F8091B40190914204980F9093F7
:1047300042042091B501280F2093B501121614F4FC
:104740009B301CF081958093B401DF91CF911F9134
:104750000F910895BF92CF92DF92EF92FF920F9345
:104760001F93CF93DF93FC01828180FF03C0DD2480
:10477000DA9402C0DD24D3940FEA13E0C0E0D0E065
:104780002FE2B22EF80111821082128294E0E92EFB
:10479000F12CC12C809141048C0D80332CF06B2DB9
:1047A0000E941D2E892F02C087FD815D082E000CFE
:1047B000990BC817D90791F480913F048E9DA001F1
:1047C0008F9D500D11245595479555954795980106
:1047D00060913E0480913D040E948710CD0CF1E071
:1047E000EF1AF108B9F621960D5F1F4FCF32D105B0
:1047F00049F60E94EA0F8091410491E0D91206C067
:10480000811102C08EE207C0815005C090E0019680
:10481000BE010E943F2E80934104DF91CF911F91F2
:104820000F91FF90EF90DF90CF90BF900895EF929F
:10483000FF921F93CF93DF93EC018FEAE82E83E082
:10484000F82E10E08C81970140913F0460913E0466
:10485000810F0E9487101B5F83E0E80EF11C1B3E56
:1048600089F70E94EA0F9A818C8190FF02C08F5FC6
:1048700001C081508C83DF91CF911F91FF90EF9009
:1048800008950F931F93CF93DF9300D01F92CDB75E
:10489000DEB78C018091430481110AC09E012F5F15
:1048A0003F4F4FEF6FEF0E9487108A818093430440
:1048B000F8018481813051F028F0823061F4409118
:1048C00043040AC08091430440E007C06091430460
:1048D00040E080E003C040E080E060E00E94201003
:1048E000F801848190E0019663E070E00E943F2E21
:1048F00084830F900F900F90DF91CF911F910F91B4
:104900000895CF93DF93EC01ECE3F4E043816281FF
:104910008C810E941D118C818F5F8C83DF91CF91E0
:104920000895CF93DF93EC01EC81F0E0EC5BFB4F5B
:104930004491ECE3F4E0628181810E941D118C813D
:104940008F5F8C83DF91CF9108952091E4003091A7
:10495000E50095E64091EC00842F817040FF23C074
:104960008091E80080FD1DC080915203882399F05A
:10497000853099F08091EB0085FD11C04091E400F5
:104980005091E5002417350729F3915011F09A0151
:10499000E1CF84E0089582E0089583E0089581E006
:1049A000089580E008954091E80042FFDDCF08952A
:1049B0008091540387FF11C08091E80082FD05C0FB
:1049C000809152038111F8CF11C08091E8008B775C
:1049D0000BC080915203882349F08091E80080FF4A
:1049E000F8CF8091E8008E778093E8000895982FA3
:1049F000973068F59093E900981739F07091EC00C2
:104A00002091ED005091F00003C0242F762F50E04C
:104A100021FD02C09F5FECCF3091EB003E7F3093D1
:104A2000EB003091ED003D7F3093ED003091EB00D5
:104A300031603093EB007093EC002093ED005093C5
:104A4000F0002091EE0027FDE5CF80E008958F7003
:104A50008093E90081E0089520915A0330915B032F
:104A60002617370748F06115710539F42091E800E1
:104A70002E772093E80001C0B901FC0120E0611508
:104A8000710579F1809152038823F1F18530F1F1BC
:104A90008091E80083FD3CC08091E80082FD2EC03B
:104AA0008091E80080FFEBCF2091F3008091F2002D
:104AB00090E0922B6115710551F08830910538F422
:104AC00021912093F100615071090196F3CF21E00B
:104AD000089709F020E08091E8008E778093E80045
:104AE000CECF2111CFCF0AC080915203882361F02D
:104AF000853061F08091E80083FD0AC08091E80074
:104B000082FFF2CF80E0089582E0089583E0089567
:104B100081E0089578941F920F920FB60F9211249E
:104B20008F939F93AF93BF9380914E0490914F04C6
:104B3000A0915004B09151040196A11DB11D809324
:104B40004E0490934F04A0935004B0935104BF912E
:104B5000AF919F918F910F900FBE0F901F9018955E
:104B60009C014FB7F89480914E0490914F04A0910E
:104B70005004B09151044FBF821B930B08952FB77F
:104B8000F89480914E0490914F04A0915004B091FC
:104B900051042FBF08951F920F920FB60F92112448
:104BA0008F939F93AF93BF9380914D04811113C056
:104BB00080914E0490914F04A0915004B091510403
:104BC0004196A11DB11D80934E0490934F04A09374
:104BD0005004B0935104BF91AF919F918F910F906A
:104BE0000FBE0F901F9018952091B3012223C9F09A
:104BF0002091520427FF15C0262F2695269526952D
:104C00002E31C8F4FC01E20FF11D677081E090E0E5
:104C100001C0880F6A95EAF7809592818923828383
:104C20000895FC0106962281621301C0128231961A
:104C3000E817F907C1F708952091B3012223C1F0C5
:104C40002091520427FF14C0262F269526952695DD
:104C50002E3130F5FC01E20FF11D677081E090E02C
:104C600001C0880F6A95EAF79281892B82830895A3
:104C7000FC0132962FEF30E04191641789F02F3F0D
:104C800019F4411101C0232F3F5F3630A9F72F3FA0
:104C900039F0FC01E20FF11D27FDFA9562830895BA
:104CA000089520914B0430914C042817390771F076
:104CB00090934C0480934B04E0914904F0914A0492
:104CC000309721F00084F185E02D0994089520911A
:104CD0004704309148042817390771F0909348042D
:104CE00080934704E0914904F0914A04309721F001
:104CF0000680F781E02D09940895E0914904F09130
:104D00004A04309721F00190F081E02D099480E071
:104D10000895EF92FF920F93CF93DF93C42FD22F7A
:104D2000FC0182818823D1F0409346040E94BF2574
:104D3000909345048093440480E28C0F883008F0FF
:104D40006DC0C77081E001C0880FCA95EAF7DF9196
:104D5000CF910F91FF90EF900C94492A80914604D7
:104D600048134BC080914404909145040E94B025A3
:104D7000883C910508F041C0CD17C9F080E28C0F46
:104D8000883040F4C77081E001C0880FCA95EAF707
:104D90000E94422A80E28D0F883048F481E09D2FE6
:104DA000977001C0880F9A95EAF70E94492A093343
:104DB00019F0E12CF12C03C080E5E82EF12C802FB6
:104DC0000E94B32AE114F10451F08FE99FE00197AA
:104DD000F1F700C0000091E0E91AF108F3CF802F4D
:104DE0000E94532A80E28D0F8830C0F4D77081E092
:104DF00001C0880FDA95EAF70AC080E28C0F88308C
:104E000068F4C77081E001C0880FCA95EAF7DF91A6
:104E1000CF910F91FF90EF900C94422ADF91CF91A8
:104E20000F91FF90EF90089590913C0490FF04C083
:104E30009695981740F003C0811105C090E0961731
:104E400010F40C945B120C944F12882311F0FA01A9
:104E500001C0FB01099480E090E00E94672680E099
:104E600090E00E94512610921E030E94AA1BE7E9BF
:104E7000F2E086E0DF011D928A95E9F71092910237
:104E800010929002109292020C9465128F929F924F
:104E9000AF92BF92DF92EF92FF920F931F93CF9347
:104EA000DF938090780290907902A0907A02B0907F
:104EB0007B02409121035091220360912303709162
:104EC0002403842A952AA62AB72ACFE1D0E02CE031
:104ED000929F700111249CE3D92E082F10E0D50178
:104EE000C4010C2E04C0B695A795979587950A9492
:104EF000D2F780FD04C0219790F780E014C0DC9EBB
:104F0000F001DD9EF00D1124EE0DFF1DE00FF11FED
:104F1000EE0FFF1FE651FF4F859194910E94871974
:104F2000019749F38C2FDF91CF911F910F91FF9043
:104F3000EF90DF90BF90AF909F908F900895CF93A8
:104F4000DF93EC010E9446272CE3829FC0011124CD
:104F5000FC012CE0D29FE00DF11D1124EC0FF11D9E
:104F6000EE0FFF1FE651FF4F859194910E94871924
:104F7000DF91CF910895FC01808191810E949F274C
:104F800092959F70963079F010F4925001C09A502B
:104F9000923068F4803F69F018F4883E40F409C00C
:104FA000843F29F406C0883E20F0813F11F080E064
:104FB000089581E008959F92AF92BF92CF92DF92C1
:104FC000EF92FF920F931F93CF93DF93CDB7DEB78E
:104FD00061970FB6F894DEBF0FBECDBF8C0185E0A0
:104FE000F801DE011D9601900D928A95E1F7F80116
:104FF000E2809091C5026091C6024091C802509132
:10500000C9024115510531F06F3F31F481E09F3FF6
:1050100019F403C081E001C080E0F82FF1709F2EE9
:1050200080FD1AC1F80130812181C380D48085ECD4
:10503000A82E82E0B82EF090C702F601E41BF50B13
:10504000FF2009F4C6C08091CA02E83CF10508F0CF
:1050500091C0482F407F09F050C0621311C09313D4
:105060000FC0FE2CE1100CC08F7080618093CA02CB
:10507000C5010E9484038091CA02F801858329C179
:10508000CD2831F02F3F31F481E03F3F19F403C0C8
:1050900081E001C080E080FD03C081E08E2502C078
:1050A00080E090E0F82FF170FF2E80FF1CC080910F
:1050B000FC024091CB0256E0841709F4E8C090E06E
:1050C000589FF001599FF00D1124E453FD4F618169
:1050D000261306C06081631303C06281E61203C019
:1050E00001968770E9CFFE2CEE2009F4F2C0809182
:1050F000CA0281608093CA0249C0621306C093133A
:1051000004C0E11002C0F80186C0C8010E94BB279C
:10511000882351F1EE2041F12091CA02822F82951D
:105120008F7090E0029774F08091C5029091C60252
:1051300098878F831986DB86CA862C87CE010796CF
:105140000E94840386E0F801A5ECB2E001900D9284
:105150008A95E1F70E94431C0AC06217C9F0C80192
:105160000E94BB2781111EC0C8010E948403FF2436
:10517000F394AFC0482F407F81F785EC92E00E9406
:10518000840386E0F50111928A95E9F7F12CA1C01C
:105190009313E5CFE110E3CFF8018583C8010E94A6
:1051A000840354C0EE2001F32091CA02822F82951D
:1051B0008F7090E0029734F28091C5029091C60200
:1051C0009A8389831B82DD82CC822E83CE01019655
:1051D000B7CFE83CF105D0F5FE2CEE2029F26213A2
:1051E00027C0931325C02091CA0220FD18C0822F2A
:1051F00082958F70482F50E04115510581F0F801DC
:1052000025834F30510541F08F5F982F9295907F05
:10521000822F8F70892B8583C8010E94840386E0CA
:10522000F801A5ECB2E001900D928A95E1F751C02A
:10523000C8010E94BB27811185CF8091CA0281607D
:105240008093CA02C8010E94840343C086E0F5012E
:1052500011928A95E9F73DC0EE2009F485CFC80187
:105260000E94BB27F82E882309F47ECF86E0F80140
:10527000A5ECB2E001900D928A95E1F78091C5020C
:105280009091C6020E949F270E94431C22C03D8726
:105290002E878D859E850E949F27292F22952F700E
:1052A000223028F49F7039F0811105C00BC02430E2
:1052B00028F49F7049F4805E883020F0C8010E9475
:1052C00084039F2CF92C05C0F8019581907F99F7F4
:1052D000F9CF8F2D61960FB6F894DEBF0FBECDBF0C
:1052E000DF91CF911F910F91FF90EF90DF90CF90C2
:1052F000BF90AF909F9008952CE0929F800D112455
:10530000682F669566956695982F977085E0689FDB
:10531000B001112440E050E080E0FB01E40FF51FF4
:10532000E95AFB4F208130E0092E02C036952795BF
:105330000A94E2F721703327042E01C0220F0A9449
:10534000EAF7822B4F5F5F4F4530510531F70895E3
:105350002CE0929F800D1124E82FE695E695E695C6
:10536000877051E001C0550F8A95EAF785E0E89F04
:10537000F0011124E95AFB4F20E030E070E0408159
:10538000CB01022E02C0969587950A94E2F78170B0
:10539000819584278523842781932F5F3F4F253074
:1053A000310569F7089560937802709379028093CC
:1053B0007A0290937B020C942B270F931F9341E06A
:1053C00050E060E070E004C0440F551F661F771F77
:1053D0008A95D2F7409550956095709580917802A6
:1053E00090917902A0917A02B0917B028A019B018F
:1053F000082319232A233B23C901B8011F910F91C8
:105400000C94D3290F931F9341E050E060E070E0CB
:1054100004C0440F551F661F771F8A95D2F78091ED
:10542000780290917902A0917A02B0917B028A0170
:105430009B01082B192B2A2B3B2BC901B8011F916B
:105440000F910C94D32960932103709322038093CE
:105450002303909324030C942B2710921F03809115
:10546000B301882331F08091520487FF02C08EE19E
:1054700001C086E0E7EAF2E0DF011D928A95E9F7D4
:105480000C942B27882321F00E94A31B0C94AA1BA9
:105490000895882339F090911F03892B80931F036F
:1054A0000C94AA1B0895882309F45CC0823869F41F
:1054B0000E947D2681FF56C069E385EA92E00E9442
:1054C0001C260E94AA1B69E30EC0833891F40E9437
:1054D0007D2680FF47C063E585EA92E00E941C2696
:1054E0000E94AA1B63E585EA92E00E94F4250C94D1
:1054F000AA1B843869F40E947D2682FF33C067E4CA
:1055000085EA92E00E941C260E94AA1B67E4EBCF6A
:105510009CEF980F913A10F4682FE5CF90E2980F26
:10552000983050F4877091E001C0990F8A95EAF79E
:10553000892F0E94A31BDBCF9BE5980F933020F4AB
:1055400080E090E00C94672698E5980F973120F45E
:1055500080E090E00C9451268D3E20F00E948F1246
:105560000C9465120895CF93882309F4BEC0C82F08
:105570008238B1F40E947D2681FDB7C069E385EAD7
:1055800092E00E941C260E94AA1B2FEF81EE94E05D
:10559000215080409040E1F700C0000069E317C04F
:1055A0008338E1F40E947D2680FD9FC063E585EA93
:1055B00092E00E941C260E94AA1B2FEF81EE94E02D
:1055C000215080409040E1F700C0000063E585EA8B
:1055D00092E00E94F425CF910C94AA1B8438B1F478
:1055E0000E947D2682FD81C067E485EA92E00E94E8
:1055F0001C260E94AA1B2FEF81EE94E021508040D0
:105600009040E1F700C0000067E4E1CF8CEF8C0F21
:10561000813AC0F58091B3018823E1F08091520472
:1056200087FF18C0EC2FE695E695E695F0E0EB5580
:10563000FD4F8281282F30E04C2F477081E090E0B1
:1056400002C0880F991F4A95E2F782239323892B82
:1056500061F412C0E7EAF2E08DEA92E02191C2170C
:1056600021F08E179F07D1F707C06C2F85EA92E0D3
:105670000E94F4250E94AA1B6C2F85EA92E00E94EA
:105680001C26A9CF80E28C0F883068F4C77081E0B7
:1056900090E001C0880FCA95EAF790911F03892B0B
:1056A00080931F0398CFEBE5EC0FE33040F4F0E07C
:1056B000EF5DFD4F808190E0CF910C946726E8E587
:1056C000EC0FE73150F4F0E0EE0FFF1FEC5DFD4F03
:1056D00080819181CF910C945126CD3E30F08C2F5A
:1056E0000E944813CF910C946512CF910895809138
:1056F000A401811122C01092AE030E94A313109244
:1057000068031092690310925D0310925C03EEE649
:10571000F3E080E090E0A0E8BFEB1182108282838A
:105720009383A483B58317821682389623E0EE3ADA
:10573000F20799F781E08093A401089562E070E098
:1057400087EC91E00E94F11C2FEF81EE94E0215054
:1057500080409040E1F700C000000E94772B6091EC
:105760006B036E7F60936B0387E090E00C94242CB6
:1057700060916B03616060936B0387E090E00E942F
:10578000242C62E070E087EB91E00C94F11C809196
:105790006A03811144C080E090E00E941E2C893E83
:1057A0009E4F11F00E94321B87E090E00E94102C67
:1057B00080936B03EEE6F3E080E090E0A0E8BFEBBF
:1057C0001182108282839383A483B5831782168209
:1057D000389623E0EE3AF20799F780916A03811137
:1057E0000CC00E94A313259A82E0809380008AE176
:1057F0008093810081E080936A030E94772B8091DF
:105800006B0380FF06C060E070E08FE794E00E94C9
:10581000F11C0E94BF2590935F0380935E0308955F
:10582000F999FECF92BD81BDF89A992780B5089568
:10583000A6E1B0E044E050E00C944A2CA8E1B0E0CE
:1058400042E050E00C944A2C262FF999FECF92BDED
:1058500081BDF89A019700B4021639F01FBA20BD35
:105860000FB6F894FA9AF99A0FBE08950396272F67
:105870000E94252C0E94242C252F0E94252C242FA9
:105880000C94252C0196272F0E94252C0C94242C57
:10589000DC01CB01FC01F999FECF06C0F2BDE1BDF0
:1058A000F89A319600B40D9241505040B8F70895DF
:1058B0000E943B2D08F481E008950E94712C0C9405
:1058C000762D0E946F2D58F00E94682D40F029F42B
:1058D0005F3F29F00C945F2D51110C94AA2D0C946C
:1058E000652D0E94872D68F39923B1F3552391F319
:1058F000951B550BBB27AA2762177307840738F03F
:105900009F5F5F4F220F331F441FAA1FA9F335D09B
:105910000E2E3AF0E0E832D091505040E695001C4F
:10592000CAF72BD0FE2F29D0660F771F881FBB1F09
:10593000261737074807AB07B0E809F0BB0B802DE7
:10594000BF01FF2793585F4F3AF09E3F510578F013
:105950000C945F2D0C94AA2D5F3FE4F3983ED4F392
:10596000869577956795B795F7959F5FC9F7880FE7
:10597000911D9695879597F90895E1E0660F771F39
:10598000881FBB1F621773078407BA0720F0621BCA
:10599000730B840BBA0BEE1F88F7E09508950E94F5
:1059A0008F2D88F09F5798F0B92F9927B751B0F0F5
:1059B000E1F0660F771F881F991F1AF0BA95C9F793
:1059C00014C0B13091F00E94A92DB1E008950C945B
:1059D000A92D672F782F8827B85F39F0B93FCCF30E
:1059E000869577956795B395D9F73EF49095809510
:1059F000709561957F4F8F4F9F4F0895E89409C030
:105A000097FB3EF490958095709561957F4F8F4FF1
:105A10009F4F9923A9F0F92F96E9BB279395F69507
:105A2000879577956795B795F111F8CFFAF4BB0F85
:105A300011F460FF1BC06F5F7F4F8F4F9F4F16C0E9
:105A4000882311F096E911C0772321F09EE8872F73
:105A5000762F05C0662371F096E8862F70E060E02F
:105A60002AF09A95660F771F881FDAF7880F9695A8
:105A7000879597F90895990F0008550FAA0BE0E84C
:105A8000FEEF16161706E807F907C0F01216130600
:105A9000E407F50798F0621B730B840B950B39F440
:105AA0000A2661F0232B242B252B21F408950A26A6
:105AB00009F4A140A6958FEF811D811D089597F9E6
:105AC0009F6780E870E060E008959FEF80EC0895A4
:105AD00000240A94161617061806090608950024CD
:105AE0000A9412161306140605060895092E039447
:105AF000000C11F4882352F0BB0F40F4BF2B11F4BB
:105B000060FF04C06F5F7F4F8F4F9F4F089557FD19
:105B10009058440F551F59F05F3F71F04795880F1B
:105B200097FB991F61F09F3F79F0879508951216B2
:105B300013061406551FF2CF4695F1DF08C016165E
:105B400017061806991FF1CF86957105610508940F
:105B50000895E894BB2766277727CB0197F9089526
:105B60000E94C32D0C94762D0E94682D38F00E945F
:105B70006F2D20F0952311F00C945F2D0C94652D62
:105B800011240C94AA2D0E94872D70F3959FC1F3C8
:105B9000950F50E0551F629FF001729FBB27F00DDB
:105BA000B11D639FAA27F00DB11DAA1F649F662730
:105BB000B00DA11D661F829F2227B00DA11D621F7F
:105BC000739FB00DA11D621F839FA00D611D221F39
:105BD000749F3327A00D611D231F849F600D211D1D
:105BE000822F762F6A2F11249F5750409AF0F1F0A0
:105BF00088234AF0EE0FFF1FBB1F661F771F881F09
:105C000091505040A9F79E3F510580F00C945F2DB4
:105C10000C94AA2D5F3FE4F3983ED4F386957795D4
:105C20006795B795F795E7959F5FC1F7FE2B880FAE
:105C3000911D9695879597F9089587FB082E06265E
:105C400087FD819567FD61950E94AC2E0EF49195BC
:105C500007FC81950895AA1BBB1B51E107C0AA1F31
:105C6000BB1FA617B70710F0A61BB70B881F991FFD
:105C70005A95A9F780959095BC01CD01089597FBA1
:105C8000072E16F4009407D077FD09D00E942B2E22
:105C900007FC05D03EF4909581959F4F089570952F
:105CA00061957F4F0895A1E21A2EAA1BBB1BFD012F
:105CB0000DC0AA1FBB1FEE1FFF1FA217B307E407EB
:105CC000F50720F0A21BB30BE40BF50B661F771F43
:105CD000881F991F1A9469F7609570958095909523
:105CE0009B01AC01BD01CF010895EE0FFF1F059090
:105CF000F491E02D09940E94832E332312F48A1B21
:105D00009B0B0C94942EA29FB001B39FC001A39F44
:105D1000700D811D1124911DB29F700D811D1124E4
:105D2000911D08950E94832EB7FF0895821B930B47
:105D300008950E94832EA59F900DB49F900DA49F5F
:105D4000800D911D11240895B7FF0C94992E0E9487
:105D5000992E821B930B0895991B79E004C0991F1B
:105D6000961708F0961B881F7A95C9F780950895B5
:105D7000FC014150504030F001900616D1F73197A8
:105D8000CF010895882799270895FB01DC0104C0FD
:105D90008D910190801921F441505040C8F7881B23
:085DA000990B0895F894FFCF60
:105DA80000005C44000080415C978A440000804108
:105DB80052D0A444000080410000DC44000080412F
:105DC80000005C440000004100005C440000004109
:105DD80000005C440000004100005C4400000041F9
:105DE80048F176440000C04000005C440000C04018
:105DF80048F176440000C04000005C440000C04008
:105E080048F176440000C04000005C440000C040F7
:105E180048F176440000C04000005C440000C040E7
:105E280052D02445000000410000DC44000000413D
:105E380052D0A4440000404102225822392235227F
:105E4800312201220101191A1B1C1D1E1F202122AB
:105E58000106000101020100005C4400000041004D
:105E680000DC44000000410000DC44000000410068
:105E7800005C440000004133323130C69734366646
:105E880067F6F7949293959600FF0100010000FFD2
:105E9800FF0000010001FF0090F091F100010202F3
:105EA80002020606060909090909090F0F0F0F0F53
:105EB8000F15151518191919191919191919192357
:105EC80024818283E200E900EA00B500B600B70049
:105ED800CD008301CC008A019201940121022302A2
:105EE80024022502260227022A02B300B4006F000A
:025EF800700038
:00000001FF
